:020000040800F2
:1000000000180020175C0008C55B00088D5C000824
:10001000C95B0008CB5B0008CD5B00080000000056
:10002000000000000000000000000000CF5B00089E
:10003000D15B000800000000D35B00084D0E0008F3
:10004000D75B0008D95B0008DB5B0008DD5B0008BC
:10005000DF5B0008E15B0008E35B0008E55B00088C
:10006000E75B0008E95B0008EB5B0008ED5B00085C
:10007000EF5B0008F15B0008F35B0008F55B00082C
:10008000F75B0008F95B0008FB5B0008FD5B0008FC
:10009000FF5B0008015C0008035C0008055C0008C9
:1000A000075C0008095C00080B5C0008D10E000822
:1000B0000F5C0008115C0008135C0008155C000868
:1000C00082B0002301930093304A116880235B02C1
:1000D0000B431360110080229202A020C0010B6824
:1000E00013400093019B01330193009B002B02D12D
:1000F000019B8342F3D1254B1B689B0339D5244BCD
:1001000011221A60214A5368F0218B435360214B1E
:100110001B68102B2FD0042B32D01C4B5A685A600E
:100120001A4B5A685A605A681B490A405A60596803
:10013000882252030A435A601968802252040A43F3
:100140001A601900802292040B681342FCD00F4BF6
:100150005A6803218A435A605A6801390A435A602F
:1001600019000C224B681340082BFBD1074B0122CE
:100170001A6302B07047536840390B435360CFE7AE
:10018000024A536890210B435360C9E700100240B4
:0C01900000200240E4140020FF7FC0FFAC
:10019C00114B1B68002B0FD10F4B32221A600F4BE7
:1001AC001B68012B0DD90E4B1B68002B05D0013B96
:1001BC000B4A1360002B00D070470A4B01229A6146
:1001CC00FAE7002B04D1074B802252029A61F3E725
:1001DC00044B01229A61EFE75815002060150020AE
:0801EC00641500200004004826
:1001F40010B5054B1860002805D01C00FFF7CCFF94
:0C0204002368002BFAD110BD6815002003
:1002100010B504F02DFC154B1A68D34301321BD0E6
:10022000FF22110019401A4217D0114A11601B0217
:100230001B0E16D00F4A13600E4B1A680E4B1A6035
:100240000E4B1968CA43FF23180088430C49086005
:10025000120C13400B4A136010BD054A0B211160AC
:10026000E5E7044B0A221A60E6E7C046006400088E
:100270007015002004150020C81400200464000834
:080280005C1500206015002050
:1002880010B544490122CB681A42FCD1414B1B6985
:100298001B0604D53F4B404A5A60404A5A603D4BC2
:1002A8001A6902210A431A613D4A5A611A693E31A4
:1002B8000A431A6119000122CB681A42FCD1354B56
:1002C800DB689B0604D5334AD36820210B43D360EF
:1002D800304B1A6902218A431A611A6901390A43A3
:1002E8001A61304B1B68DB432D4A138029490122D0
:1002F800CB681A42FCD1274BDB689B0604D5254AFC
:10030800D36820210B43D360274B1B68DB43274A64
:10031800138020490122CB681A42FCD11D4BDB68AF
:100328009B0604D51B4AD36820210B43D360204B7E
:100338001B68DB431F4A138016490122CB681A4207
:10034800FCD1144BDB689B0604D5124AD3682021E4
:100358000B43D360184B1B68DB43184A13800D49C5
:100368000122CB681A42FCD10A4BDB689B0604D5F4
:10037800084AD36820210B43D360064B1A69012130
:100388008A431A611A697F310A431A610A20FFF702
:100398002DFF10BD0020024023016745AB89EFCD3A
:1003A800006400087015002004150020026400088D
:1003B8005C1500200464000860150020066400082D
:1003C800F8B5C34B1C68631E012B00D915E2C1495F
:1003D8000122CB681A42FCD1BE4B1B691B0604D50F
:1003E800BC4BBD4A5A60BD4A5A60BA4A13690221D9
:1003F8000B431361012C00D1C4E0B64BB84A5A61D3
:10040800B44A136940210B43136111000122CB68E0
:100418001A42FCD1AF4BDB689B0604D5AD4AD368C2
:1004280020210B43D360AB4B1A6902218A431A611E
:100438001A6901390A431A61013C63425C4164420A
:10044800A84B1C40A64B9C466444A74B1B68013331
:10045800DB4323809F490122CB681A42FCD19D4B84
:10046800DB689B0604D59B4AD36820210B43D360E5
:100478009E4B1B68DB43638096490122CB681A4276
:10048800FCD1944BDB689B0604D5924AD3682021A3
:100498000B43D360964B1B68DB43A3808D49012235
:1004A800CB681A42FCD18B4BDB689B0604D5894A82
:1004B800D36820210B43D3608E4B1B68DB43E3805A
:1004C80084490122CB681A42FCD1824BDB689B0627
:1004D80004D5804AD36820210B43D360864B1B6820
:1004E8001B02864A12781343DB4323817949012290
:1004F800CB681A42FCD1774BDB689B0604D5754A5A
:10050800D36820210B43D3607D4B1B68DB43638199
:1005180070490122CB681A42FCD16E4BDB689B06FE
:1005280004D56C4AD36820210B43D360754B1B68F4
:100538001B02DB43A38167490122CB681A42FCD125
:10054800644BDB689B0604D5624AD36820210B43C1
:10055800D3606D4B1B68DB43E3815E490122CB68A6
:100568001A42FCD15B4BDB689B0604D5594AD36819
:1005780020210B43D36010346448564B01222025B8
:10058800634E07E01300634A5A6139E704340430C4
:10059800B04219D00168C9432180D9680A42FCD108
:1005A800D9680D4202D0D9682943D9600168C94386
:1005B800090C6180D9680A42FCD1D9680D42E5D09E
:1005C800D9682943D960E1E7424B1A6901218A4376
:1005D8001A611A6901310A431A613D4B1C68012CE2
:1005E8002DD03C4B4C4A5A613A4A136940210B437F
:1005F800136111000122CB681A42FCD1354BDB682C
:100608009B0604D5334AD36820210B43D360314B72
:100618001A6902218A431A611A6901390A431A615F
:10062800013C63425C4164422E4F27403A4B9C4652
:1006380067443C00274B01222025384E07E0254B14
:10064800374A5A61D0E704340430B04219D00168FF
:10065800C9432180D9680A42FCD1D9680D4202D029
:10066800D9682943D9600168C943090C6180D968F0
:100678000A42FCD1D9680D42E5D0D9682943D9602E
:10068800E1E780239B009C4667442648114B0122E2
:100698002025254E03E004370430B04246D00168D7
:1006A800C9433980D9680A42FCD1D9680D4202D0C1
:1006B800D9682943D9604188C9437980D9680A42F1
:1006C800FCD1D9680D42E6D0D9682943D960E2E760
:1006D8005C1500200020024023016745AB89EFCD5F
:1006E8000074000800F4FFFF6015002004150020C6
:1006F80048150020E4140020D8140020E01400203D
:10070800DC14002000150020381500200408002003
:10071800F40B00200068000800780008F40D0020A1
:10072800006C00080402002004040020334B1A69FE
:1007380001218A431A611A6901310A431A61304B4F
:100748001C68012C2CD02D4B2E4A5A612B4A136958
:1007580040210B43136111000122CB681A42FCD1DE
:10076800264BDB689B0604D5244AD36820210B431B
:10077800D360224B1A6902218A431A611A69013926
:100788000A431A61013C63425C4164421E4B1C40AF
:100798001C4B9C466444194B012220251B4E07E044
:1007A800164B1B4A5A61D1E704340430B04218D0C2
:1007B8000168C9432180D9680A42FCD1D9680D4231
:1007C80002D0D9682943D9604188C9436180D96872
:1007D8000A42FCD1D9680D42E6D0D9682943D960CC
:1007E800E2E7064B1A6901218A431A611A697F31C7
:1007F8000A431A610A20FFF7F9FCF8BD00200240FD
:100808005C150020007C000800F4FFFF04080020AD
:040818000070000864
:10081C00304A91698023DB010B4393619022D2050E
:10082C0013682D490B401360116880239B030B4305
:10083C0013602A4B19682A480140196018688021F6
:10084C00890101431960516A264801405162506A7E
:10085C0080214900014351621A6A23490A401A62F5
:10086C001A6A1A62214B224A1360224A1360224BE5
:10087C001B68392B29D01ED8132B28D0263B5A1E87
:10088C0093415B421D4A13401D4A944663441D4AE2
:10089C00938180239B025360002393602C3313605D
:1008AC00136801210B431360174B1960174B8022FF
:1008BC0012051A607047603B5A1E93415B42144A02
:1008CC001340144A94466344E1E7134BDFE7134BA0
:1008DC00DDE7C04600100240FFFFEFFF00040048B8
:1008EC00FFEFFFFFFFF0FFFFFFFFFFF014110020F1
:1008FC00501500204C15002070150020BFFCFFFF88
:10090C00E2040000003801406C15002000E100E01A
:10091C0019EEFFFF8813000041030000C40900001A
:10092C000A498022CB691A42FCD080B2074B188549
:10093C00074B1B68032B00D07047064B80225202DA
:10094C009A61054B04221A60F6E7C0460038014054
:0C095C0060150020000400486415002015
:10096800F0B5C64600B5494B1B68002B65D0013B66
:100978005A4253415B42464C1C40464B9C46644499
:100988002068C3436168CA430140013100D16EE069
:100998001904090C0139404801601B0CFF210B4068
:1009A8003E4803603E480360130C0B403D490B6012
:1009B800012B04D0102B02D00B0001211960120466
:1009C800120C394B1A60A368DB439A05920F37491A
:1009D8000A603F221A4036490A601B0C354A1360E8
:1009E800E368DE4325001035370C334B1F603F01A9
:1009F8002C4B1B6898461900380005F081FB2F4BDB
:100A0800186033041B0E7E2B01D901235B422C4A4C
:100A1800136047452ED22B4A2B4908CDDB4308C229
:100A28008A42FAD1C023DB009C466444274A2848FE
:100A380008CCDB4308C28242FAD103F04BFE1A4BC2
:100A48001B68002B07D09023DB051B8A5B0502D4AB
:100A5800154B00221A600D20FFF764FF01F0C4F95E
:100A6800114B1B68002B0AD180BCB846F0BD03F0BF
:100A7800FBFFE2E702F04AFA02F0BEFACBE7013BDD
:100A8800144A136003F032FBEEE7C0465C15002001
:100A980000F4FFFF00740008601500200415002012
:100AA800C8140020E414002048150020D8140020A1
:100AB800E0140020DC140020381500201C1500204C
:100AC8000015002004080020F40D00200402002076
:080AD80004080020FC140020BA
:100AE00070B5041E00DA9CE0092C00D893E0632C5A
:100AF00000D881E0FA239B009C426ED3534B9C426A
:100B00005AD9534B9C4248D9524B9C4236D9524BEE
:100B10009C4224D9514B9C4212D9514B9C4200D942
:100B200084E05049200005F0EFFA05004D4920000F
:100B300005F04FFA0C0028003030C0B2FFF7F6FE87
:100B40004949200005F0E0FA05004749200005F07A
:100B500040FA0C0028003030C0B2FFF7E7FE4349EE
:100B6000200005F0D1FA05004049200005F031FAD7
:100B70000C0028003030C0B2FFF7D8FE3C492000FE
:100B800005F0C2FA05003A49200005F022FA0C00EF
:100B900028003030C0B2FFF7C9FE3649200005F00A
:100BA000B3FA05003349200005F013FA0C002800C1
:100BB0003030C0B2FFF7BAFEFA218900200005F0FC
:100BC000A3FA0500FA218900200005F002FA0C00C2
:100BD00028003030C0B2FFF7A9FE6421200005F0E4
:100BE00093FA05006421200005F0F3F90C002800B9
:100BF0003030C0B2FFF79AFE0A21200005F084FAD7
:100C000005000A21200005F0E4F90C00280030302E
:100C1000C0B2FFF78BFE20003030C0B2FFF786FE77
:100C200070BD2D20FFF782FE64425DE7124920006F
:100C300005F06AFA05001049200005F0CAF90C0019
:100C400028003030C0B2FFF771FE6AE70F270000BE
:100C50009F8601003F420F007F969800FFE0F50558
:100C6000FFC99A3B00E1F5058096980040420F00CD
:0C0C7000A08601001027000000CA9A3B7B
:100C7C00F8B5454D454C02E06420FFF7B5FA444BFE
:100C8C005969802292020A435A6159698022D20220
:100C9C000A435A619021C90500260E603D4B1E6027
:100CAC003D4ACA60DA60DA680327BA43DA601A6828
:100CBC00BA431A6019680122114319609A612A60BB
:100CCC00FFF7F8F9354B1E60354B1E60354B1E6037
:100CDC00354B0B221A60354B1E600A23344A1360C5
:100CEC00344A1360344B1F60344B354A1A602B68FE
:100CFC005901C91A8900C918C900324B186805F086
:100D0C00FDF9013880235B0498420DD22E4A5060C5
:100D1C002E48036A1B021B0AC02109060B430362FF
:100D2C0000239360073313603220FFF75DFA03F062
:100D3C00CFFCFFF767FA0220FFF756FAFFF768FDC2
:100D4C000220FFF751FA0D20FFF7EAFD204804F0CE
:100D5C00DAFF3220FFF7E4FD2E20FFF7E1FD0B2038
:100D6C00FFF7B8FE1B4804F0CEFFFFF7F7FD03F0CA
:100D7C0017FD02F007FA002800D17DE72368002B4D
:100D8C00F5D003F015FAF2E7E4140020BC140020AF
:100D9C000010024000040048AAAAAAAA6415002068
:100DAC006815002054150020701500206C150020CB
:100DBC0004150020C814002060150020F014002039
:100DCC00A1B0B9120002002010E000E000ED00E03C
:080DDC00A85C00088C5400081B
:100DE40010B5FFF7D9F9114B1B68114A12689342E9
:100DF40019D05A1C0D490A601B7880200002184340
:100E04000C4B1B689A420BD00B4B1B68012B06D969
:100E14000A4B802252029A61094B04221A6010BDC7
:100E2400084A0A60F0E70020F9E7C0464C150020A4
:100E340050150020FC01002060150020000400482B
:080E44006415002014110020C8
:100E4C00194B1B68002B02D0013B174A1360174B40
:100E5C001B68002B02D0013B144A1360144B1B6817
:100E6C00002B02D0013B124A1360124B1B68002B63
:100E7C0002D0013B0F4A13600F4B1B68002B02D0B2
:100E8C00013B0D4A13600D4B1B68002B02DD013B2F
:100E9C000A4A13600A490A6853035A40530C5340D8
:100EAC005A0153400B6070475815002068150020FC
:100EBC005415002010150020CC140020E81400203C
:040ECC00F0140020FE
:100ED00010B5114BDB699B0612D50F4B9B8C99B259
:100EE000FF221340022B0CD0042B12D00B4A1368A4
:100EF0001970136801331360094A1268934204D0D1
:100F000010BD084BFD3A1A60F0E7044B064A1A6020
:100F1000F6E700F095FDF3E700380140501500209A
:0C0F2000FC010020C0140020141100206F
:100F2C00024A202311680B431360704724150020DC
:100F3C00064A1368043B1360054A0C32934204D2F0
:100F4C00044A042311680B4313607047EC1400200F
:080F5C00881300202415002079
:100F6400084B1A68111D1960074B6033994202D26D
:100F7400136853607047054A042311680B431360D8
:100F8400F8E7C046EC140020881300202415002044
:100F9400044B19680A1F1068096811601B681860FF
:080FA4007047C046EC14002068
:100FAC00034A1368191D11601A1F12685A607047A2
:040FBC00EC14002011
:100FC000074A1368190008390868043B1B680B605E
:100FD0001368191F1B680B60136818607047C046C0
:040FE000EC140020ED
:100FE400074A13681968181F006818601368181FE7
:100FF400083B1B6803601368083B19607047C046D0
:04100400EC140020C8
:101008000C4B19680A680C4BCB1A9B109B1A042BC3
:1010180006D4002A0AD092008A1A13680B60704717
:10102800064A042311680B431360F8E70439014B9F
:101038001960F4E7EC140020881300202415002020
:1010480030B5144B1A681168134BD31A9B105B1AEE
:10105800042B19D4043A0F4B1A60012913D9012320
:101068005B1A9B009D580222521A9200094C236871
:1010780098589B18043B1860013904320029F6D1AE
:10108800044B1B681D6030BD044A042311680B43E0
:101098001360F8E7EC1400208813002024150020C2
:1010A800F0B5144B1A681568134BD31A9B105B1BC9
:1010B800042B19D4043A17680E4B1A60012D12D963
:1010C8006E1E0422524200211C00236898589B1867
:1010D80058600131043AB142F7D101235D1B054B39
:1010E8001B68AD00EF50F0BD044A042311680B43A0
:1010F8001360F8E7EC140020881300202415002062
:10110800054B1A68111F12680868844662440A6011
:0C1118001A68043A1A607047EC140020BA
:10112400024B1A681368013313607047EC140020F3
:10113400054B1A68111F12680868821A0A601A6837
:0C114400043A1A607047C046EC1400200A
:10115000024B1A681368013B13607047EC140020BF
:10116000044B1A681368002B00DB70475B42136066
:08117000FBE7C046EC1400206F
:1011780010B50F4B1B681A68D117501848401F2824
:1011880009DC191F0A4C2160002A0BDB0B000968D7
:101198009140196010BD074A8023DB0011680B439A
:1011A8001360F7E7043B1A68C2401A60F2E7C046CA
:0811B800EC14002024150020B6
:1011C000054B1A68111F1268086802400A601A6805
:0C11D000043A1A607047C046EC1400207E
:1011DC00054B1A68111F1268086802430A601A68E6
:0C11EC00043A1A607047C046EC14002062
:1011F800054B1A68111F1268086842400A601A688D
:0C120800043A1A607047C046EC14002045
:10121400024B1A681368DB4313607047EC14002018
:10122400024B1A6813685B4213607047EC14002089
:10123400054B1A68111F1268086842430A601A684D
:0C124400043A1A607047C046EC14002009
:1012500010B50B4B1C682168002909D0043C20689C
:1012600004F034FF2060064A1368043B136010BD8D
:10127000044A80231B0111680B431360F7E7C04643
:08128000EC14002024150020ED
:1012880010B50B4B1C68216800290AD0221F106872
:10129800083C23685843064B1C6004F013FF206089
:1012A80010BD044A80231B0111680B431360F7E744
:0812B800EC14002024150020B5
:1012C00010B50B4B1C682168002909D0043C20682C
:1012D00004F02EFF2160064A1368043B136010BD22
:1012E000044A80231B0111680B431360F7E7C046D3
:0812F000EC140020241500207D
:1012F80070B50D4B1C682568002D0ED0043C26687F
:101308002900300004F010FF2160074B1C682900F9
:10131800300004F0D7FE206070BD044A80231B0112
:1013280011680B431360F7E7EC1400202415002024
:101338000B4B1B681A681F2A0BD8043B01219140EC
:101348000A0019680A431A60054A1368043B1360C7
:101358007047044A8023DB0011680B431360F7E7EA
:08136800EC1400202415002004
:101370000B4B1B681A681F2A0AD8043B01219140B5
:101380001A688A431A60064A1368043B1360704760
:10139000044A8023DB0011680B431360F7E7C04663
:0813A000EC14002024150020CC
:1013A8000C4B1B681A681F2A09D8012191400A00B2
:1013B800191F0968114209D001221A6005E0064A7E
:1013C8008023DB0011680B431360704700221A600A
:0C13D800FBE7C046EC14002024150020A8
:1013E400034A1368191D1160024A12685A60704753
:0813F400EC140020F0140020AD
:1013FC00064A1368191F1B6808681B1A5842434198
:10140C000B601368043B13607047C046EC1400205B
:10141C00064A1368191F1B6808681B1A581E83415B
:10142C000B601368043B13607047C046EC1400203B
:10143C00034B1A6811684B424B4113607047C0460E
:04144C00EC1400207C
:10145000074B1A68131F012112681868904200DCBC
:1014600000211960024A1368043B13607047C046AC
:04147000EC14002058
:1014740030B5074B1A68111F10680A68D217C40FD9
:101484000D68854262410A601A68043A1A6030BDE8
:04149400EC14002034
:10149800074B1A68131F012112681868904200DB75
:1014A80000211960024A1368043B13607047C04664
:0414B800EC14002010
:1014BC00064A1368191F1B68086884469C459B41A3
:1014CC005B420B601368043B13607047EC14002004
:1014DC0030B5074B1A68111F08681468C20FE5175E
:1014EC0084426A410A601A68043A1A6030BDC046E8
:0414FC00EC140020CC
:10150000114B1A681368002B0CD0C82B0ADC190089
:10151000C83107DB002B0CDD013B9B000B495B58FE
:10152000136005E00A4A8023DB0011680B43136057
:101530007047DB439B00111F086804495850083A64
:10154000014B1A60F4E7C046EC140020F40D0020B3
:04155000241500203E
:10155400044B0A221A60044B1B68002B01D1034B75
:101564001A607047C81400202815002004150020B4
:10157400044B10221A60044B1B68002B01D1034B4F
:101584001A607047C8140020281500200415002094
:1015940005490A681368043A0A60002B02D0013B2B
:0C15A400002BFCD17047C046EC14002066
:1015B00004490B6864221868424303480260043BF4
:0C15C0000B607047EC140020CC140020DD
:1015CC0010B5054B1C68221D1A60044B1868642169
:1015DC0004F094FD606010BDEC140020CC140020CD
:1015EC0030B5094B1B68013B08495B181B041C0CEC
:1015FC00074802681B0E15684B5513689C466144DE
:10160C004C70043A026030BD3415002004020020F6
:04161C00EC140020AA
:10162000044B1A68111D1960034B1B68043B1B68AF
:0C16300053607047EC140020F4140020FC
:10163C00024B1B681A68024B1A607047F4140020A6
:04164C00181500204D
:10165000064B1B681A68002A04D1054A12681168F3
:10166000044A1160043B014A13607047EC140020E7
:08167000F414002018150020FD
:10167800154B1B68154A19681160154A934218D909
:10168800144A1268022A07D0043B0F4A1360124A10
:101698001368013B136070470F4A11680F4A1268BC
:1016A8009142F1D10D4A002111600A4A03311160BB
:1016B800EAE7064B00221A60064B1B68022BEAD1A8
:1016C800044B03321A60E6E7F414002018150020D2
:1016D80018130020F80100200C15002044150020E4
:1016E800054B00221A605A609A6018000C300349B2
:1016F8000860DA607047C04688130020EC140020A8
:0C170800014B03221A607047F80100201A
:0C171400014B01221A607047F801002010
:0C172000014B00221A607047F801002005
:10172C0030B50D4B1C68221D1A600C490B685A1CF5
:10173C000A60587800069A1C0A609A7812040243D0
:10174C00D81C0860D87800021D1D0D601B7913434E
:10175C000343636030BDC046EC1400201815002014
:10176C00054A1368191D116004490A68501C086069
:10177C0052785A607047C046EC14002018150020AF
:10178C00074B19680A1D1A60064A1368581C10602A
:10179C005A781201044B9B189B684B607047C046EB
:0C17AC00EC140020181500200408002098
:1017B800074B1A68511C19600648036851780901DB
:1017C800054A521819689160043B03607047C04687
:0C17D80018150020EC140020040800206C
:1017E400074B1A68511C196051780902901C186043
:1017F40092781143802292050A431A607047C046CA
:041804001815002093
:1018080010B5094B1868021D1A6008490B685A1C64
:101818000A605A7812029C1C0C609B781A43802339
:101828009B051343436010BDF414002018150020D5
:10183800074B1A68511C196051780902901C1860EE
:1018480092781143802292050A431A607047C04675
:04185800181500203F
:10185C0010B5094B1B681A68023A80239B05134389
:10186C001A78742A03D1013B044A136010BD034A51
:10187C001360FFF7DBFFF9E7F414002018150020C4
:10188C0010B50A4B1B681B68002B0CD0084A136858
:10189C00043B1360074A136803331360034A13684D
:1018AC00043B136010BDFFF7C1FFF7E7EC140020F9
:0818BC00F414002018150020AF
:1018C40010B50A4B1B681B68002B0CD1084A13681F
:1018D400043B1360074A136803331360034A136815
:1018E400043B136010BDFFF7A5FFF7E7EC140020DD
:0818F400F41400201815002077
:1018FC0010B5104B1A681100103119600E490B68A5
:10190C00180008380068D060181F006890601868CC
:10191C0050600C3B0B6009480368591C01605978F6
:10192C0009029C1C04609B78194380239B050B4384
:10193C00136110BDF4140020EC14002018150020C5
:10194C00204B1B681A1F12681900083908680439E3
:10195C000968521800291ADB904210DD043B1A600A
:10196C00194B1A68511C196051780902901C1860A7
:10197C0092781143802292050A431A607047103BFB
:10198C00104A1360104A136803331360F6E7904251
:10199C0010DA043B1A600C4B1A68511C1960517810
:1019AC000902901C186092781143802292050A4318
:1019BC001A60E3E7103B034A1360034A13680333CE
:0C19CC001360DBE7F41400201815002065
:1019D800024A1368043B13607047C046F4140020A1
:1019E800024A1368103B13607047C046F414002085
:1019F80008490B681A6808480260043B0B60032A10
:101A080000D87047054A8023DB0011680B43136038
:101A1800F7E7C046EC1400206015002024150020CC
:101A280010B5044C23681878FEF77CFF2368043B44
:081A3800236010BDEC14002036
:101A400010B50F4B1B68002B00D010BD2020FEF7F7
:101A50006DFF2D20FEF76AFF3E20FEF767FF442052
:101A6000FEF764FF4220FEF761FF4720FEF75EFFAE
:101A70002020FEF75BFF024B01221A60E5E7C0461B
:041A8000F801002049
:101A840070B50A490A68561C0E6054783619002C41
:101A940009D00D002B685A1C2A605878FEF744FFC1
:101AA400013C002CF6D1014B1E6070BD18150020BE
:101AB40010B5114B1B68002B12D0104B1B68002B68
:101AC4000ED00F4B1B68002B15D00E4A1368191D3E
:101AD40011600D4A12785A60094B00221A600AE01C
:101AE400FFF77EF90028FBD0064B1A68111D196018
:101AF400FF231840506010BDF8010020201500207D
:0C1B0400C4140020EC1400207415002014
:101B100010B50E4B1B68102B08D00D4B1B681868B6
:101B2000E0231B06C2180B4B9A420CD8084B1B68CB
:101B3000186804F0BFFA2020FEF7F8FE044A136884
:101B4000043B136010BDFEF7CBFFF4E7C814002080
:081B5000EC140020FF0B06302D
:101B580010B5064C2368186804F0A8FA2020FEF790
:101B6800E1FE2368043B236010BDC046EC1400204E
:101B7800F0B587B003AA2A4B13CB13C2294B1A68B6
:101B880001929A8801AB9A805B20FEF7CBFE264B28
:101B98001B68264A0C3293420DD0244A0C329342D9
:101BA8000DD3224A0C32934216D9204C1034042506
:101BB8001E4F160024E001A804F0A7F80CE003A8C3
:101BC80004F0A3F8194B00221A605A609A601800B2
:101BD8000C3015490860DA605D20FEF7A3FE20206E
:101BE800FEF7A0FE07B0F0BD206804F05FFA2020E1
:101BF800FEF798FE01350C4B1B680434B342EBD951
:101C0800DB1B9B10AB42E7D32020FEF78BFE084B73
:101C18001B68102BE8D02068FEF75EFFE7E7C04698
:101C2800E45C0008F05C0008EC1400208813002035
:041C3800C8140020AC
:101C3C00F0B5D6464F464646C0B584B001AA394BDE
:101C4C0003CB03C21B7813702020FEF769FE364BC2
:101C5C001B68002B5BD0354D00270026C0231B05CD
:101C6C009946334B9A46304B984616E02020FEF7A7
:101C7C0057FE14E06B684A46134221D12020FEF730
:101C8C004FFE2020FEF74CFE01360137052F34D8CD
:101C9C00103543461B68B34237D9092EE6D93000BC
:101CAC00FEF718FF3A20FEF73BFE2C00083C20788C
:101CBC000028DFD0FEF734FE0134AC42F7D1D9E76F
:101CCC0001A804F020F853461B68102B11D028688B
:101CDC00FEF700FF2020FEF723FE4020FEF720FE3B
:101CEC002804000C04F0E0F92920FEF719FE023755
:101CFC00C4E7286804F0D8F9ECE70D20FEF710FED5
:101D0C002020FEF70DFE0027C2E7002F05D104B0FE
:101D1C00E0BCBA46B146A846F0BD0D20FEF700FE69
:101D2C00F5E7C046BC5E0008081500200C08002032
:041D3C00C8140020A7
:101D400010B5044C2368186804F089F82368043B34
:081D5000236010BDEC1400201B
:101D5800F0B5C64600B582B06846214B020012CBEA
:101D680012C203F0D2FF0D20FEF7DCFD1D4DFA2351
:101D78009B009846A8440026012723E0FEF7D2FDE1
:101D88000134285D0028F9D1062C05D82020FEF75B
:101D9800C9FD0134072CF9D12320FEF7C3FD380013
:101DA80003F0DDFF2020FEF7BDFD2020FEF7BAFD81
:101DB8002020FEF7B7FD01370136052E07D008357C
:101DC800A84509D02020FEF7ADFD0024D9E70D2055
:101DD800FEF7A8FD0026F2E702B080BCB846F0BDC9
:081DE800A4540008DC570008B8
:101DF00070B5A8B0DB4B1A6826929A8869469C2079
:101E000009180A809B796A469E215218137023ACE8
:101E1000D54B220023CB23C221AAD44B1968219190
:101E2000998891809B7993711FAAD14B03CB03C2F0
:101E30001CAAD04B03CB03C211001A880A809B78DE
:101E40008B7019AACC4B23CB23C215AACB4B23CB27
:101E500023C21B78137012AAC94B03CB03C21B8881
:101E600013800FAAC74B03CB03C21B8813800DAA94
:101E7000C54B03CB03C20AAAC44B03CB03C21B78D6
:101E80001370C34B099307AAC24B03CB03C2C24BC7
:101E90001A6805929A8805AB9A8002AABF4B03CBB9
:101EA00003C21B7813706A46BD4B03CB03C24420A8
:101EB000FEF73CFD6120FEF739FD7420FEF736FD8C
:101EC0006120FEF733FD26A803F023FFB5480C3050
:101ED00004F094F85220FEF729FD6520FEF726FD58
:101EE0007420FEF723FD26A803F013FFAE4804F08C
:101EF00085F8200003F00DFFAC4804F07FF8552072
:101F0000FEF714FD7320FEF711FD6520FEF70EFDB0
:101F10007220FEF70BFD3D20FEF708FDA44804F0FB
:101F20006DF80D20FEF702FDA24B1B68002B00D1BF
:101F3000D9E01FA803F0EDFE9E4B1B68002B00D0DC
:101F4000D5E01CA803F0E5FE9B4B1B680024002B8A
:101F500000D1D6E0964E984D2B68013B1B01F3183B
:101F6000185D002804D0FEF7E1FC0134082CF3D101
:101F700019A803F0CEFE914B186830231843C0B265
:101F8000FEF7D4FC15A803F0C4FE8D4D8D4E3268CB
:101F90005101891A8B01591AC900891889012868C9
:101FA00004F0B2F80400FEF79BFD2E20FEF7BEFC05
:101FB00033685A01D21A9100C918C900286804F080
:101FC000A3F863011B1B9B001B19DB00C01AFEF763
:101FD00087FD4D20FEF7AAFC4820FEF7A7FC7A20DB
:101FE000FEF7A4FC0D20FEF7A1FC12A803F091FE61
:101FF000754C2068FEF774FD23680B2B00D18DE033
:10200000714B1B68132B00D18FE06F4B1B68262B85
:1020100000D18EE06C4B1B68392B00D18DE0302055
:10202000FEF784FC3020FEF781FC684B1B68002B18
:1020300000D186E02020FEF779FC2020FEF776FC18
:102040005320FEF773FC5020FEF770FC4920FEF78A
:102050006DFC3D20FEF76AFC5D4B1868FEF740FD05
:102060002C20FEF763FC5B4B1B68102B00D16CE04F
:10207000594B1868FEF734FD2C20FEF757FC574BE0
:102080001868FEF72DFD0DA803F043FE544B1B68A6
:10209000002B00D0A8E00020FEF722FD0AA803F0E4
:1020A00038FE504B1868002800DADBE0494B1B680B
:1020B000102B00D1DAE0FEF713FD07A803F029FE8C
:1020C0003B4B9B6C013300D0D7E09023DB059B8A10
:1020D000DB0700D5CDE0684603F01BFE0D20FEF7C0
:1020E00025FC28B070BD21A803F013FE21E72320B2
:1020F000FEF71CFC2F4B18683030C0B2FEF716FC00
:102100001FE76E20FEF712FC6F20FEF70FFC6E201B
:10211000FEF70CFC6520FEF709FC29E73520FEF7E9
:1021200005FC3220FEF702FC6AE73220FEF7FEFBD8
:102130006BE73420FEF7FAFB6CE73620FEF7F6FB80
:102140006DE70FA803F0E5FD74E7234B186803F073
:10215000B1FF2C20FEF7EAFB204B186803F0AAFF22
:1021600091E7C046AC540008B4540008C0540008BD
:10217000C8540008D0540008DC540008E854000893
:10218000F8540008045500081055000818550008B8
:102190004F464600245500082C55000834550008C9
:1021A0004055000888130020181300200402002066
:1021B000040800205C150020481500206015002050
:1021C00000020020E4140020701500206C1500208F
:1021D000D8140020C8140020E0140020DC140020D3
:1021E0001C150020001500202B4B1E68642575432C
:1021F00029002A4803F088FF0400FEF771FC6643BB
:10220000B3059B1B9C01A4196400A419E400244B92
:102210009C4664442E20FEF789FB2900200003F031
:1022200073FFFEF75DFC2900200003F0D2FE8C0056
:10223000641864002900200003F066FF06002900EE
:10224000200003F0C6FE880040184000290003F07B
:102250005BFF042383429B415B42F6183000FEF78C
:102260003FFC1BE709A803F054FD26E703F022FF1B
:1022700023E72D20FEF75AFB2DE705A803F049FDC3
:10228000084B1868FEF72CFC02A803F042FD064B31
:10229000986CFEF725FC21E738150020C0C62D00FC
:0C22A00080C3C901D014002004080020F5
:1022AC0010B588B001A91F4B0A0013CB13C213CB76
:1022BC0013C21B6813601C4A13681C68043B136030
:1022CC00112C17D0192C28D0382C0FD12624132CD4
:1022DC0014D0262C12D0392C10D0602C0ED0134ACE
:1022EC008023DB0011680B43136014E0572C02D1E0
:1022FC00392403E00B24962C10D1602401A803F0A0
:10230C0002FD0D20FEF70CFB094B1C60FDF7B6FF20
:10231C00084B00221A6008B010BD13240B2CEDD012
:10232C00D5E7C04648550008EC14002024150020C1
:08233C00701500206C15002053
:1023440070B5FEF74DFD041E00D1D7E0C0B26F4B4F
:102354001B68002B08D06E4B1B68002B04D06D4B00
:1023640018706D4B01221A600A2800D1C3E00228BC
:1023740000D8C2E0664B1C68002C08D109281ED086
:10238400664B1B683F2B02D9202800D19DE02828EA
:1023940017D02F283FD01B2867D1002C00D1ADE0E7
:1023A4000E38FEF7C1FA5D4B1A685D4B2021995433
:1023B4009B18002159705B4B1A6002249EE0173071
:1023C400DEE7594B1C68002C01D0002496E0FEF790
:1023D400ABFAFEF705FD0028FBD0C0B220280BD0D5
:1023E4004E490B684E4A2825D554D21850700233F2
:1023F4000B60FEF799FA81E0484B1B6801334A4AA7
:1024040013601838FEF790FA2020FEF78DFA0820A2
:10241400FEF78AFA72E0444B1C68002C01D00024B9
:102424006CE0FEF781FAFEF7DBFC0028FBD0C0B2BB
:102434002F280BD039490B68394A2F25D554D21887
:10244400507002330B60FEF76FFA57E0334B1B6892
:102454000133354A13602738FEF766FA2020FEF769
:1024640063FA0820FEF760FA48E0092848D01228E9
:1024740048D0082817D12C4B1D680024002D3DD1CD
:10248400264B1C68002C39D0013C1C60244B2022B4
:102494001A55FEF749FA2020FEF746FA0820FEF7FF
:1024A40043FA2C002AE00D2817D11C4B1B68002B83
:1024B4000BD11A4B1A681A4B202199549B180021EE
:1024C4005970184B1A60012418E0174B1B68012B34
:1024D400EFD00D20FEF728FAEBE7134B1C68002C15
:1024E40012D10E4D0E4B2A689854FEF71DFA2B6834
:1024F40001332B6002E0002400E00024200070BDC2
:102504000324FBE70424F9E70024F7E7F80100209B
:102514002015002074150020C4140020B8140020D5
:0C252400F8130020BC1400202C1500202F
:1025300010B5154B1968154B5A5C202A09D14B1C54
:102540001248013819000133C25C202AFAD00E4B20
:1025500019600023002A10D00C4840180C4CC25CB3
:10256000202A03D01A5501330F2BF8D1084A002036
:10257000D0545B18074A136010BD054B00221A7037
:10258000044B1960F8E7C046AC140020F813002093
:082590005C140020B8140020C7
:10259800F0B5DE46474680B587B00E0002AA002493
:1025A80005E0002B1BD001340132102C08D0035D4C
:1025B8001370190061391929F3D8203B1370F2E719
:1025C800002302AAD37313782D2B0ED1254B00229A
:1025D8001A6001239B460127012C0FD82CE0002309
:1025E80002AAD37313782D2B2CD01E4B00221A600D
:1025F80000239B4600270120002C2DD0194B1D6875
:10260800B84602AB9C46E044002301934346187841
:10261800310003F034FC431C18D075432D180137E2
:1026280001239C46E0440193A742EFD30D4B1D6064
:1026380001205B46002B0FD00A4A13685B421360E7
:10264800012009E00020012CC0D105E0019B002BEE
:1026580001D0044B1D60002007B0C0BCBB46B0468B
:08266800F0BDC046B0140020D3
:1026700010B5344B187800285AD000233149013363
:102680005A5C002AFBD12D280FD0302829D12D4AA1
:10269000527820218A43582A11D02B4A11681029D8
:1026A0003AD1082B48D900204BE0012B3AD0264ADA
:1026B000116810292AD00B2B3ED9002041E0214A75
:1026C00092782D2A09D00A2B2ED81E4810210230CC
:1026D000FFF762FF431E984133E00B2BF5D9002032
:1026E0002FE02528D9D1174A52782D2A09D00B2B53
:1026F0001CD814480A210130FFF74EFF431E9841B1
:102700001FE00C2BF5D900201BE000232D28C8D199
:10271000092B11D9002014E02D28CCD000200A2B41
:102720000FD809E000200CE000200AE0002008E0BB
:10273000054B19681029E8D00248FFF72DFF431E0A
:0C274000984110BD5C140020C81400205B
:10274C00F0B51A4C00251A4E0021635C8A5D180006
:10275C00613819280DD8203BDBB2100061381928DC
:10276C0011D8203AD2B2934219D101310829ECD1B7
:10277C0015E01000613819280DD918002038471EB3
:10278C00B84140420340934209D1002AEDD1094B94
:10279C001D600120F0BD203AD2B2202BE3D10135CF
:1027AC0008347E2DD0D10020F4E7C046D457000861
:0827BC005C140020FC14002055
:1027C40070B51A4B1B78002B29D0194A00231E0020
:1027D400013310321100103909780029F7D1731C24
:1027E4001FD03301114C1C19124D16E08B4211D12C
:1027F40000290BD00132082A0CD0A15C535D1800CB
:1028040061381928F2D8203BDBB2EFE70A4B1E608F
:10281400012070BD103C013E05D30022EDE70020ED
:10282400F7E70020F5E70020F3E7C046040800209E
:0C283400140800205C140020FC1400209C
:1028400010B50F4B1A680F4B1A60FFF771FEFFF7B8
:10285000B9FF002805D00C4B1B6801330B4A1360ED
:1028600010BD0B4B1B78302B05D00A4A2123116871
:102870000B431360F4E7054B00221A60F0E7C046F3
:10288000B8140020AC140020FC14002048150020CF
:082890005C1400202415002057
:10289800074A13680749C85401331360064A93422C
:1028A80004D9064A202311680B4313607047C046B9
:1028B8003415002004020020FE0500002415002025
:1028C80010B5144B18688200134BD3581A030AD456
:1028D800124A1268002A13D19B030BD48000104BB4
:1028E800C358984705E00F4A80239B0011680B43A3
:1028F800136010BD0B4A082311680B431360F8E7F7
:10290800DB0304D58000064BC3589847F1E7FFF76F
:10291800BFFFEEE7FC140020DC5500082815002056
:0829280000000020241500202E
:1029300070B594B00CA9414B0A0013CB13C213CB52
:1029400013C203CB03C205A93D4B0A0013CB13C22C
:1029500013CB13C21B7813706A463A4B13CB13C2C6
:1029600011001A680A601B790B71374B1B68522BD8
:1029700009D95224354E344DA05DFDF7D7FF0134FF
:102980002B68A342F8D85223314A1360314A002100
:102990001160314A13602E4D304E03E02C4B1A6803
:1029A0002D4B1A60284C2B682268934234D2FFF7D3
:1029B000BFFD3378002BF6D0FFF75AFE00280BD06E
:1029C000274B1A68274B1A60274B1B68002BE5D052
:1029D000264B01221A60E1E7FFF7B8FE002811D06C
:1029E000234B1B689B00234A9B585B0321D5FFF7B1
:1029F0006BFF214B1B68002B08D1154B1A68164B37
:102A00001A60CFE70CA803F084F905E01A4B002206
:102A10001A60684603F07DF90D20FDF787FF522309
:102A2000094A13600A4A13600A4B00221A6014B064
:102A300070BD05A803F06DF9EEE7C046D45E00084E
:102A4000F45E0008105F0008BC140020F81300209A
:102A5000B81400202C150020AC1400205C140020B9
:102A6000B01400203C150020201500204015002047
:0C2A7000FC140020DC5500082415002098
:102A7C0070B56E20FFF70AFF0C4D2C68FF20FFF796
:102A8C0005FFFF20FFF702FF2B68013B084A9B184C
:102A9C001B04180C074909681B0E0D6853550B686D
:102AAC009C46624450700C6070BDC04634150020CA
:082ABC0004020020EC140020CC
:102AC40010B56F20FFF7E6FE064A1368191D116062
:102AD400054A12685A60FF20FFF7DCFEFF20FFF76B
:0C2AE400D9FE10BDEC14002034150020B9
:102AF00010B57320FFF7D0FE064A1368191D116048
:102B0000054A12685A60FF20FFF7C6FEFF20FFF754
:0C2B1000C3FE10BDEC14002034150020A2
:102B1C00F8B57420FFF7BAFE104E33681D68013506
:102B2C000F4C2D19280AFF273840FFF7AFFE38004D
:102B3C002840FFF7ABFE0B4B1B68013B1B1932689F
:102B4C00190A106821541268A41863707620FFF7D4
:102B5C009DFE3368043B3360F8BDC046EC14002086
:082B6C000402002034150020D2
:102B740010B5234B1B68002B17D1224B1B68224A2C
:102B840019681160214A93422ED9214A1268022AF7
:102B94001DD0043B1B4A13601E4A1368013B13609B
:102BA4001D4B1A681D4B1A6010BD6420FFF772FE9E
:102BB4000022134B1A601A490B6801330B601B0186
:102BC40018495A54184B1A68184B1A60E8E7114A06
:102BD4001168174A12689142DBD1154A002111602D
:102BE4000B4A03311160D4E7074B00221A60084BEB
:102BF4001B68022BD4D1064B03321A60D0E7C046BF
:102C040028150020F41400201815002018130020A3
:102C1400F80100200C15002004150020C814002021
:102C24000815002004080020341500203015002069
:042C34004415002023
:102C380070B5324B1B68002B27D1314B1B681C78B1
:102C480023005F3B022B16D97D20FDF76BFE202069
:102C5800FDF768FEFEF78CFF25006F3D072D15D99F
:102C6800733C012C1CD9032D0FD8264B1B681888E0
:102C780003F0E6F909E0244B186801300005000D5F
:102C880003F0DEF92920FDF74DFE70BD2020FDF789
:102C980049FE5220FDF746FE3A20FDF743FEDFE7E6
:102CA800184B1A68194BD31A082BEED90C3A10880E
:102CB80003F0C6F92020FDF735FE2020FDF732FE8F
:102CC800104C2368083B188803F0BAF92020FDF758
:102CD80029FE6920FDF726FE2368043B188803F0C7
:102CE800AFF92020FDF71EFE7820FDF71BFE2368B4
:102CF8001888013003F0A4F9C7E7C046241500205E
:102D080014150020F41400201815002018130020B2
:102D1800084B1868084B1B68984208D001D2181A4B
:102D28007047C01A80239B009C466044F8E7002047
:0C2D3800F6E7C0464C15002050150020A6
:102D440010B5094B1C68221D1A60084B1B68002B28
:102D540006D0074B1B68002B02D0064B186801E015
:102D6400FFF7D8FF606010BDEC140020F8010020CC
:082D740020150020C41400200A
:102D7C0010B50B4B1C6800230A4909190A48CA5C98
:102D8C00222A03D01A5401334F2BF8D1064A2221A0
:102D9C00D15401330021D154E318044A136010BDFF
:102DAC00AC140020F81300205C140020B814002090
:102DBC001A4B1B185A781300613B192B03D8203A75
:102DCC001300373B05E02F2A1BD91300303B092B8E
:102DDC00F6D80F2B18D8114A1018827811006139C7
:102DEC00192907D8203A373A11000F2912D818019F
:102DFC00401870472F2A0AD9110030390929F4D903
:102E0C00F1E701204042F4E701204042F1E70120C4
:102E1C004042EEE701204042EBE7C0465C14002044
:102E2C0070B5324B1B680133314A1360FFF7A0FFBA
:102E3C00002600242F4A03E001360134502C0ED01A
:102E4C00A35C5C2BF8D0222BF7D12A4B00221A550D
:102E5C00294B1D68002D08D1264C260032E0274A4C
:102E6C00022311680B4313603EE06520FFF70EFD53
:102E7C00234A13687600A41B2249CC5401331360F7
:102E8C0000241C4D2E0005E0FFF700FD0134335DDE
:102E9C00002B29D0285D5C28F6D12000FFF788FF95
:102EAC00431C03D00334FFF7F1FCF0E7134A022371
:102EBC0011680B43136017E0FDF732FD0135735DAC
:102ECC00002B11D0605D5C28F6D12800FFF770FF55
:102EDC00431C04D00335C0B2FDF722FDEFE7074ACF
:102EEC00022311680B43136070BDC046B814002058
:102EFC00AC1400205C1400202815002024150020A0
:082F0C0034150020040200202E
:102F140070B52F4B1C6824012E4B1D68290020001E
:102F240003F0F0F82C4B186080235B02984227D3FF
:102F3400294B2A4A1A602A4B1B88DB0710D4284BDA
:102F440000221A821A802749CA6902200243CA61F0
:102F5400254A1A836422DA621A8801210A431A80F4
:102F64001D4B1B68013B9BB21D4A13851F4B1B68FD
:102F7400002B27DB1A4A138C01210B43138420E016
:102F8400AC42D8D2164A13880124A34313800023E9
:102F940017490B6017490B60144B01214942196012
:102FA4009023DB051868144D28401860D96829401F
:102FB400D960D868802189010143D960138CA34367
:102FC400138470BD138C01218B431384F9E7C0462D
:102FD40038150020E41400201C150020FFFF000019
:102FE4000004004000100240606000000015002052
:0C2FF400B4140020F8140020FFCFFFFFF1
:103000009022D205136827490B401360264A138C7F
:1030100001218B431384254B1B68002B22DB90215D
:10302000C905CA681F480240CA60002B22D0632B22
:103030002ADC9023DB051968802292010A431A607A
:103040001A6A1B490A401A62196A802252040A430A
:103050001A62154B1A8C01210A431A84134A12680A
:103060005A6370479022D205D16880239B010B439D
:10307000D360F6E70B000968802252010A431A6008
:103080008022D2039A61ECE7084B64221A609023F5
:10309000DB051968802252010A431A6040229A61B6
:1030A000DFE7C046FFCFFFFF00040040001500200F
:0430B000FFFFFFF02F
:1030B400324B9B6C002B60DD314A1268002A29DBFD
:1030C40030490A60304A1268022A1ED008DC002AFD
:1030D4000ED0012A45D19022D205022191610FE040
:1030E400032A3ED19022D2058021890291613EE0DB
:1030F4009022D20580214902916180218902916147
:1031040021490A6801320A6034E09022D205012183
:103114009161F5E752421B490A601B4A1268022A70
:103124001AD008DC002A0ED0012A1AD19022D20526
:1031340001219161E4E7032A13D19022D205802171
:103144004902916113E09022D205802149029161E4
:10315400802189029161D3E79022D20502219161F5
:10316400CEE709490A6801320A60032A02DD064AE9
:1031740000211160013B014A936470470408002058
:0C318400D0140020E8140020D414002017
:1031900070B500230D4A13600D4A13600D4A136089
:1031A0000D4C0E4D0E4E03E0FFF7CCF800280BD16E
:1031B000A36C002BF8D02B68002BF5DD3368002BB7
:1031C000F2D1FFF777FFEFE7012070BDB8140020C0
:1031D000BC1400202C15002004080020D01400206E
:0431E000E8140020CF
:1031E40070B522490B681A6821480260043B0B60E1
:1031F400002A39D01F4C204D204E0FE0204B1B6875
:10320400022B19D01F4B1B68002B03D01E4B1B68CD
:10321400002B15D1164B1B68002B25D0FCF7BCFFE7
:10322400A36C002BEAD02B68002BE7DD3368002B5E
:10323400E4D1FFF73DFFE1E7114B00221A6013E0F0
:10324400FFF77EF8012806D0022807D00F4B1B6831
:10325400002BDFD008E0FFF769FBF7E70B4A802378
:103264005B0011680B43136070BDC046EC14002072
:103274001015002004080020D0140020E8140020B9
:10328400C0140020F801002020150020241500207F
:1032940010B5044B1A68642311684B431360FFF79D
:0832A4009FFF10BDEC14002097
:1032AC00094A13681868043B136018280BD90300EB
:1032BC00A03B182B05D9054A8023DB0011680B4372
:1032CC0013601F2318407047EC14002024150020B5
:1032DC0010B5FFF7E5FF104B1B68002B0FD10F2823
:1032EC000ED89023DB051B8A0122824013400B4928
:1032FC000A68101D0860002B0AD00123536010BD12
:10330C00074B1B8A0F2210400E3A82401340EEE707
:10331C0000235360F3E7C04624150020EC14002072
:04332C000004004851
:10333000062800D07047074B1B680133FAD0064AB5
:10334000138C01218B431384024B012252421A60D9
:0C335000F0E7C04600150020000400401B
:10335C0070B5FFF7A5FF0400204B1B68002B18D19C
:10336C000F281CD80A2815D0FFF7DCFF60000322B9
:10337C0082409023DB05D9689143D9601968914349
:10338C0019601D6801221100814029431960A24077
:10339C009A6170BD114B8022D2001A60F9E70423A8
:1033AC0002009A43122A13D0103C60000322824080
:1033BC000B4BD9689143D9601968914319601D680A
:1033CC0001221100814029431960A2409A61E0E773
:1033DC00024B8022D2001A60DBE7C0462415002085
:0433EC000004004891
:1033F00070B5FFF75BFF0400214B1B68002B19D150
:103400000F281DD80A2816D0FFF792FF600003226C
:1034100082409023DB05D9689143D96019689143B4
:1034200019601D6801221100814029431960103480
:10343000A2409A6170BD124B8022D2001A60F9E757
:10344000042302009A43122A15D0010010394900C2
:1034500003228A400B4BD8689043D8601868904389
:1034600018601868012215008D4029000143196079
:10347000A2409A61DEE7024B8022D2001A60D9E7AF
:0834800024150020000400489F
:1034880010B5FFF70FFF04001D4B1B68002B15D16B
:103498000F2819D80A2812D0FFF746FF6400032224
:1034A800A2409023DB05196891431960D9689143BC
:1034B800D960D9680122A2400A43DA6010BD104BD6
:1034C8008022D2001A60F9E7042302009A43122AE4
:1034D80010D0103C64000322A2400A4B19689143A3
:1034E8001960D9689143D960D9680122A2400A437A
:1034F800DA60E3E7024B8022D2001A60DEE7C046BA
:08350800241500200004004816
:1035100010B5FFF7CBFE04001D4B1B68002B15D127
:103520000F2819D80A2812D0FFF702FF64000322DF
:10353000A2409023DB05196891431960D968914333
:10354000D960D9680222A2400A43DA6010BD104B4C
:103550008022D2001A60F9E7042302009A43122A5B
:1035600010D0103C64000322A2400A4B196891431A
:103570001960D9689143D960D9680222A2400A43F0
:10358000DA60E3E7024B8022D2001A60DEE7C04631
:0835900024150020000400488E
:1035980010B5FFF787FE0400184B1B68002B10D1ED
:1035A8000F2814D80A280DD0FFF7BEFE64000322A6
:1035B800A2409023DB05196891431960D9689143AB
:1035C800D96010BD0D4B8022D2001A60F9E70423A0
:1035D80002009A43122A0BD0103C64000322A24036
:1035E800074B196891431960D9689143D960E8E796
:1035F800024B8022D2001A60E3E7C046241500205F
:043608000004004872
:10360C0010B5144BDA6814490A40DA6099698022C3
:10361C0092000A439A6102F05AFB02F058FB02F046
:10362C0056FB02F054FB0D4B0022DA608021090698
:10363C001961022159610A490A609A6801210A43F9
:10364C009A60190001220B681A42FCD002F03FFB71
:10365C0010BDC04600100240FFFDFFFF00240140DA
:04366C0008270140EA
:103670000C4B1A6801210A431A609A6801310A4307
:103680009A60190001228B681A42FCD1064B9A6994
:1036900006490A409A61D968802292000A43DA609A
:1036A0007047C0460024014000100240FFFDFFFFAC
:1036B000F0B5C64600B52C4B802252029A61FFF746
:1036C000D7FF2A4BDA6801218A43DA609A690A43F4
:1036D0009A619024E4052668E26890462068244FA9
:1036E00038402060E2683A40E260E068214A0243E4
:1036F000E260214800228260026142611F4802604C
:103700001F4F4760C7601F48076904252F430761A3
:103710005D698027FF032F435F611B4F3A601B4D9C
:10372000FD60BFF34F8FBFF36F8F40BF20BF20BF3F
:1037300002615A69164802405A61DA680A43DA603F
:1037400002F0CBFAFCF7BCFC124B134A1360134A8D
:10375000136026604346E36002F0BFFA5E20FDF787
:10376000E5F880BCB846F0BD0004004800100240F7
:103770003FFFFF3F400000400000014000040140C7
:103780000884000000ED00E000140048AAAAAAAADC
:10379000FFFFBFFF14110020501500204C15002022
:1037A000F0B589B004AA5C4B13CB13C21B881380FD
:1037B0006A465A4B13CB13C21B781370584B1B68C5
:1037C0001C68621C18D0072C03D92300A03B072BD0
:1037D0001BD8544B9B699B051ED5534B534A1A600B
:1037E0000F232340590003228A40072B00D990E081
:1037F00099004F4841588F46043B494A1360FFF7F0
:1038000037FF684602F085FA35E04A4A8023DB003C
:1038100011680B4313602EE0FFF7F8FE04A802F0D6
:1038200078FADAE79021C905086810430860C8688B
:103830009043C86001229A4013003B4A93620426D9
:10384000002714000425A3682B43A36023681D42AE
:10385000FCD0236CFF1802F040FA013E002EF2D19A
:103860002F4B1B68BA081A60BB0704D52C4B1A688B
:1038700013680133136009B0F0BD9021C9050868D1
:1038800010430860C8689043C860D3E79021C90519
:10389000086810430860C8689043C860CAE7902170
:1038A000C905086810430860C8689043C860C1E74C
:1038B0009021C905086810430860C8689043C86033
:1038C000B8E79021C905086810430860C8689043AC
:1038D000C860AFE718490968013108D01748018C62
:1038E0000124A14301841449012040420860902131
:1038F000C905086810430860C8689043C86099E724
:103900009021C905086810430860C8689043C860E2
:1039100090E700238EE7C046305F0008405F000854
:10392000EC1400200010024000240140FF070000BA
:1039300064550008241500200015002000040040F4
:103940001A4B1B68032B25D8194B1B68043B1C2BF7
:1039500020D880235B02174A12689A421AD2164B6B
:103960001A6816490A401A6019688822D2000A4368
:103970001A60DA6812490A40DA60D9688022920037
:103980000A43DA60094B1B68012B0AD90A4B08224B
:103990009A6105E00B4A8023DB0011680B4313603A
:1039A0007047054B802212039A61F9E7D814002072
:1039B000E0140020DC140020000400483FF0FFFF6A
:0839C000FFFCFFFF24150020AD
:1039C80010B50A4A13680A4918680860191F116077
:1039D800086808490860190008391160086806492C
:1039E80008600C3B1360FFF7A7FF10BDEC14002024
:0C39F800DC140020E0140020D814002093
:103A0400F0B5DE4657464E464546E0B583B0454BD5
:103A14001B68A822D2001340013AFF3A93421DD1F9
:103A2400414B1C68012C1CD93E4B08229A613F4B28
:103A34001B689B461B6801933D4B19683D4B1D68F1
:103A440000220126374880239B039A462023994667
:103A540080231B03984608239C4636E0FFF76EFF3D
:103A6400DEE7304B802212039A61E0E7534683611C
:103A740033E0012C0BD92B4B083199615B461A605A
:103A840003B0F0BCBB46B246A946A046F0BD254BE8
:103A9400802109039961F1E743468361002D2FD109
:103AA4005200038A1B0933401A4304E05200038A7C
:103AB4001B0933401A43634683612B00002B02D059
:103AC400013B002BFCD10029D3D0013933008B40BA
:103AD400019F1F42CAD04B468361002C0CD0032C9B
:103AE400DAD063468361002D0AD15200038A1B0990
:103AF40033401A432B0011E043468361002DD5D097
:103B04002B00013B002BFCD15200038A1B093340DC
:103B14001A43002CCFD02B00032CCCD0474687610E
:103B2400CCE7C04600040048D8140020EC14002060
:083B3400E0140020DC14002065
:103B3C0010B5074A1368191D1160064A12685A60BD
:103B4C00FF20FEF7A3FEFF20FEF7A0FE10BDC0462F
:083B5C00EC14002034150020D8
:103B6400F8B5104E33681D6801350F4C2D19280A1D
:103B7400FF273840FEF78EFE38002840FEF78AFE05
:103B84000A4B1B68013B1B193268190A106821543F
:103B94001268A41863707520FEF77CFE3368043B3A
:103BA4003360F8BDEC14002004020020341500201A
:103BB40070B57D280DD8C0000E4D441908352D1858
:103BC4002078002804D0FCF7AFFE0134AC42F7D1D2
:103BD40070BD7F2528400001074D441908352D1874
:103BE40020780028F4D0FCF79FFE0134AC42F7D1D2
:0C3BF400EEE7C046D4570008040800208B
:103C000070B50001064D441908352D18207800289C
:103C100004D0FCF78BFE0134AC42F7D170BDC04636
:043C20000408002074
:103C2400F0B5C64600B582B0AA4B1A6800929B88CC
:103C34006A469380A84B1D68002D03D002B080BC57
:103C4400B846F0BDA54B1B68A54A13601B7898467F
:103C54001F00A44B1B685E00F6180D20FCF764FEE1
:103C6400002E06D02C002020FCF75EFE0134A64274
:103C7400F9D19B4B188802F0E5F92020FCF754FE9B
:103C8400404602F0DFF92020FCF74EFE7E2F1AD8C2
:103C94004046FFF78DFF6A2F53D06B2F57D06C2F00
:103CA40000D182E06D2F00D187E06E2F56D0702FA7
:103CB40000D18AE0712F00D18DE0FD224346723B92
:103CC40013424BD059E02D20FCF72EFE3E20FCF78A
:103CD4002BFE2020FCF728FE4046FFF769FF7F4BB0
:103CE4001B685B787F241C40682F00D19EE0692FFD
:103CF40000D1A5E0642F00D1C6E07B4C032D00D198
:103D0400D6E02368022B00D8D2E0FCF745FAFFF78F
:103D140001F80028F2D0FEF713FB0500012800D1BA
:103D2400BCE0022800D1BCE00428E7D16D4B1B683D
:103D3400002B00D1BCE06D4A13606B4B02221A6069
:103D4400DCE76B4B1B681B68002B07D0C7E7684B8D
:103D54001B68191F1A680B689A42C0D0684601F0A4
:103D6400D6FF5E4B1B68587800029B7818430130DD
:103D740002F068F92920FCF7D7FD662F35D1574B9F
:103D84001B685C782820FCF7CFFD5A4B1B68102B6E
:103D940027D02000FCF7A2FE2920FCF7C5FD4F4BDD
:103DA4001B685B787F241C40A1E7514B1B681A1FDA
:103DB40012681B689A42D1D291E74D4B1B681A1FB7
:103DC40012681B689A42C9D989E7494B1B681B686A
:103DD400002BC3D083E7464B1B681B68002BBDD167
:103DE4007DE7200002F064F9D6E7672F00D076E77C
:103DF4003A4B1A6893781B04517809060B431179DE
:103E04000B43D47824021C432820FCF78DFD394B46
:103E14001B68102B06D02000FCF760FE2920FCF75D
:103E240083FD67E7200002F043F9F7E72820FCF759
:103E34007BFD2000FFF7E2FE2920FCF775FD5CE71F
:103E44002820FCF771FD2000FFF7D8FE4020FCF786
:103E54006BFD240120000830274E80190004000C5B
:103E640002F026F92320FCF75FFD3419A068214BEA
:103E74001B68102B05D0FCF731FE2920FCF754FDFC
:103E84003BE702F015F9F8E72020FCF74DFD3C2054
:103E9400FCF74AFD2D20FCF747FD2EE7FEF746FD13
:103EA4002CE70D4A80235B0011680B431360C5E6C1
:103EB4002020FCF739FD43465F3B022B03D86846BC
:103EC40001F025FFBAE67B20FCF72EFD2020FCF74D
:103ED4002BFDB3E60C5D0008241500201815002006
:103EE400141500200C150020F801002044150020B2
:0C3EF400EC140020C8140020040800207A
:103F000010B5FFF78FFE074B1B68002B08D1064B3F
:103F10001B681B789B00054A9B589847FEF78CFE50
:103F200010BDC046241500201815002000000020F8
:103F300010B51B4A1368013313601A4B1A68111D20
:103F4000196019490B6853601A787F2313401B01CD
:103F5000164AD3189B680B601B787D2B0BD8144A2C
:103F60001268032A04D09B00124A9B58984710BD40
:103F7000FFF7C6FFFBE70E4B1B68032B06D00E4B6B
:103F80001B68002BF3D1FFF7D3FFF0E7FFF74AFEE2
:103F9000094B1B68002BEAD1FEF74EFEEFE7C04647
:103FA0000C150020F414002018150020040800202F
:0C3FB000F8010020000000202415002073
:103FBC00F0B587B001AA3F4B13CB13C211001A689E
:103FCC000A601B790B713C4B1B683C4C3C4AA41897
:103FDC00A34269D23B4D384E2F003EE0FFF7A2FFC3
:103FEC0045E0FEF793FE00280CD133681B787D2B3F
:103FFC001BD8344A1268032A14D09B00324A9B58AF
:10400C00984734E0FEF798F9012808D00228ECD143
:10401C002E4A80235B0011680B43136044E0FEF7CB
:10402C0081FCE2E7FFF766FF21E03B68032B02D03F
:10403C00FFF778FF1BE0FFF7EFFDFEF7F7FDF7E763
:10404C00224B1B68002B2FD11B4B1B68002B1DD048
:10405C000133194A1360A34226D22A68002AC0D120
:10406C001B787D2BBAD89B00174A9B589847184B46
:10407C009B6C002BE4D0174B1B68002BE0DD164B20
:10408C001B68002BDCD1FFF70FF8D9E70D4B1B6831
:10409C00032B0BD00B4B01221A6000230F4A136029
:1040AC000F4A13600F4A136007B0F0BD01A801F06E
:1040BC002AFEEFE75C5F00081815002004020020C0
:1040CC00F40D0020F8010020000000202415002031
:1040DC0004080020D0140020E81400202015002033
:0840EC00401500200C15002016
:1040F400F8B5274B1C68002C2ED1264B1B681901E0
:10410400254A5218D168C022120511420AD0234A06
:104114001168081D10601B011F4AD3189B684B606F
:104124002000F8BD1B011C4AD3189A681C4B1A6066
:104134001C4B01221A601C4D2F681C4C266852230C
:104144002B6023601A4B00221A60FFF735FF2F60A3
:104154002660184B1C68E3E70E4B186802010E4BEF
:104164009B18DA68C0231B0514001C401A4204D1B2
:1041740080231843FEF78EFBD2E76820FEF78AFB04
:10418400044B1868FEF786FB0A4B1C68C8E7C04658
:1041940028150020FC14002004080020EC14002042
:1041A4001815002020150020BC140020B81400208D
:0841B4002C1500202415002049
:1041BC0070B50023384A1360384A1360384A1360CC
:1041CC001500384E0EE0384B1B68FF2B24D86620A8
:1041DC00FEF75CFB344B1868FEF758FB304B1A6843
:1041EC002E4B1A60314C2B682268934230D2FEF76A
:1041FC0099F93378002BF6D0FEF734FA00281FD04B
:10420C002B4B1B68002BDED12A4A1368191D116039
:10421C00254A12685A60E1E76720FEF737FB224C0B
:10422C0003202056FEF732FB0223E05EFEF72EFB46
:10423C0023681812FEF72AFB2068FEF727FBCDE750
:10424C00FEF7BAFA002809D0FFF74EFF002800D07D
:10425C0070BD134B1A68114B1A60C3E7FEF770FA66
:10426C0000280AD0FEF72AFB134B1B68002BEFD15A
:10427C000B4B1A68094B1A60B4E70F4A01231168FB
:10428C000B4313600D4B1A680D4B1A60044B1A68E4
:10429C00024B1A60DCE7C04620150020AC1400204D
:1042AC00B81400205C140020B0140020BC140020B2
:1042BC0028150020EC1400202415002030150020B7
:0442CC003415002085
:1042D000F0B5DE4657464E464546E0B593B00CA9CC
:1042E000BA4B0A0013CB13C203CB03C21B78137063
:1042F00007AAB74B13CB13C211001A680A609A8839
:104300008A809B798B7103AAB24B13CB13C21B8893
:104310001380B14B1A68B14B1A60FEF709F9FEF72A
:1043200051FA00280DD1FEF711FA002805D1AC4A48
:10433000012311680B43136018E10CA801F0E9FC9C
:1043400014E1A54B1A68A54B1A6007A801F0E1FC1F
:10435000A44D2B681801A44C001901F0ABFE0D20F0
:10436000FCF7E4FA2B681A01A418E168C0221205D0
:10437000080010400190114200D0FEE01B019A4A53
:10438000D3189C68994BE41A2405240D1B5D012564
:10439000642B00D1D1E0954E24E00D20FCF7C6FA45
:1043A000019D1FE0914B1A195078000202341F5DE5
:1043B00007432820FCF7BAFA781C01F045FE2920B3
:1043C000FCF7B4FA01352020FCF7B0FA2020FCF706
:1043D000ADFA0134854B1B5D642B00D1ADE0013596
:1043E000072DDAD8A0190004000C01F02DFE3A20A8
:1043F000FCF79CFA305DFFF7DDFB335D1A006A3A8B
:104400000A2ACFD9662B1AD0672B2ED0682B4CD016
:10441000692B57D0652BD6D12220FCF787FA734B36
:104420001B195B789B46A31C98465B46002B7DD0EE
:104430006E4B434499465C460F239A466BE0013429
:104440002820FCF773FA6A4B1B68102B08D0674BC7
:10445000185DFCF745FB2920FCF768FA0135B2E747
:10446000624B185D01F026FEF5E76048021993786B
:104470001B04517809060B43D7783F020434025DD0
:1044800013431F432820FCF751FA594B1B68102B8C
:1044900007D03800FCF724FB2920FCF747FA013548
:1044A00091E7380001F006FEF6E701342820FCF71A
:1044B0003DFA4E4B185DFFF7A3FB2920FCF736FAB7
:1044C000013580E701342820FCF730FA474B1F5DA7
:1044D0003800FFF795FB3F01083743483F1840205D
:1044E000FCF724FA3804000C01F0E4FD2920FCF765
:1044F0001DFA013567E75C20FCF718FA380901F06E
:10450000FAFB5046384001F0F6FB013C01239C4683
:10451000E144002C09D04B461F783B00203B5E2B2A
:10452000E9D83800FCF702FAEFE7D8444446013CEA
:104530002220FCF7FBF9033545E72C48201800043E
:10454000000C01F081FD3A20FCF7F0F93B20FCF76C
:10455000EDF9244B1A681201234B9B18DA68C0232B
:104560001B051A4209D10D20FCF7E0F913B0F0BC8D
:10457000BB46B246A946A046F0BD03A801F0C9FB60
:104580001B4B1B68102B18D0164B1A681201164BC8
:104590009B18986801F063FC2020FCF7C7F94020C5
:1045A000FCF7C4F90F4B1868000108300E4BC01817
:1045B0000004000C01F07EFDD5E70A4B1A681201D9
:1045C000094B9B18986801F075FDE5E72C5D000824
:1045D000445D0008585D0008B8140020AC140020A9
:1045E00024150020FC1400200408002004020020F0
:0445F000C8140020CB
:1045F400134B1B68134A1360134A126812011349C0
:104604005218BE20C000844661448A420AD210492E
:104614000139891A8908013189005118002001C221
:104624008A42FCD10B4A934209D80B4A9B180B4986
:104634008C4662440021197001339342FBD17047C8
:10464400341500203015002008150020040800202F
:10465400F40D0020FE05000004020020FF05000008
:1046640010B5164B1A68164B1A60FDF75FFFFEF77C
:10467400A7F800280DD0114B1A68114B1A60114B82
:104684001B68042B0BD8104A802311680B4313605A
:1046940004E00D4A212311680B43136010BD0B4A3B
:1046A40013600B4A1B0100219954D318DB681B05C6
:1046B4001B0D084A1360FFF79BFFEFE7B8140020B7
:1046C400AC140020FC140020241500200815002040
:0846D400040800203415002049
:1046DC0010B50023204A1360204A1360204A13604F
:1046EC00204A1360204A1360204A01211160204A9D
:1046FC001360204B1A68204B1A60204A0023117853
:10470C00002903D0013310325F2BF8D11C4A1360FF
:10471C001C4A1D4BD35C642B1CD01B4B1100013B62
:10472C00CA5C642A02D0002BF9D102E0002B00D025
:10473C000133164A1360FFF757FF154A154B1A60E1
:10474C0000231360144A0F491160144A1360FCF7DC
:10475C00C5FF10BD0C4BEBE72C15002028150020D5
:10476C0020150020401500200C150020F801002019
:10477C00C414002004150020C814002004080020D4
:10478C000815002004020020FF050000341500204D
:10479C0018130020F41400201815002024150020F4
:1047AC0030B5B3B030AA984B196830919988918084
:1047BC009B7993712EAA954B19682E9199889180AB
:1047CC009B7993712BAA924B03CB03C211001A88CD
:1047DC000A809B788B7028AA8E4B13CB13C225AA08
:1047EC008D4B03CB03C211001A880A809B788B7007
:1047FC0021AA8A4B13CB13C21B8813801BA9884B8D
:10480C000A0013CB13C203CB03C21B78137017AA75
:10481C00844B13CB13C21B68136013AA824B13CBAC
:10482C0013C21B8813800EAA804B13CB13C211002A
:10483C001A680A609B888B8008A97D4B0A0013CBF1
:10484C0013C203CB03C21B78137004AA794B13CB8E
:10485C0013C21B7813706A46774B13CB13C21B8899
:10486C001380764B1A68764B60339A4200D27CE008
:10487C0074490423086803430B60714B0C339A4250
:10488C0004D2704A042311680B4313606E4B1B68EF
:10489C00002B0FD06D4B19686D4B09010022CA54C7
:1048AC005B185A709A70DA701A715A719A71DA71BF
:1048BC009A60DA60644B00221A60664B1B68002B0E
:1048CC000ED00024634D2020FCF72AF801342B680D
:1048DC00A342F8D85E20FCF723F80D20FCF720F853
:1048EC0030A801F010FA574C206801F0A7FB3D20CE
:1048FC00FCF716F82368DB075AD4524B1B689B074E
:10490C005AD4504B1B685B075AD44E4B1B681B0781
:10491C005AD44C4B1B689B065AD44A4B1B681B063B
:10492C005AD4484B1B68DB055AD4464B1B689B0575
:10493C005AD4444B1B685B055AD4424B1B681B056D
:10494C005AD42EA801F0DFF9424B1868FCF7C2F8D4
:10495C002920FBF7E5FFFFF7BBFE0D20FBF7E0FF7F
:10496C003D4B00221A6033B030BD354B0C339A42AC
:10497C0000D286E7334B1B68002B00D086E7324B06
:10498C001B68002B3CD1354B1B68012BE5D020203C
:10499C00FBF7C6FF6F20FBF7C3FF6B20FBF7C0FFD5
:1049AC002F4B1B68102BD8D14820FBF7B9FFD4E74D
:1049BC002BA801F0A8F9A0E728A801F0A4F9A0E71A
:1049CC0025A801F0A0F9A0E721A801F09CF9A0E727
:1049DC001BA801F098F9A0E717A801F094F9A0E73B
:1049EC000EA801F090F9A0E713A801F08CF9A0E74C
:1049FC0008A801F088F9A0E704A801F084F9A0E761
:104A0C00684601F080F9A8E7985D0008A05D0008F1
:104A1C00A85D0008B45D0008C05D0008CC5D00080E
:104A2C00DC5D0008F45D0008045E0008145E0008FC
:104A3C00285E0008405E0008505E0008EC14002060
:104A4C0088130020241500202815002008150020AC
:104A5C0004080020AC140020401500202C15002068
:044A6C00C81400204A
:104A700010B50023274A1360012227490A602749FD
:104A80000B6027490A60274A5168F0208143516032
:104A900051685160244A1360244A08211160244A55
:104AA0002A311160234A1360234A1360234B0122E9
:104AB00052421A60224B323256240021C020000597
:104AC0001C705A709970D860996010330132D2B25C
:104AD000352AF5D11A4B0B324E219954013205314A
:104AE0009954013201319954043901329954002208
:104AF00044201A54C0200005D86401204042986424
:104B00001048052404605A540F4B1A60FFF7E6FD65
:104B100010BDC0465C150020F8010020481500209B
:104B2000E414002000100240D8140020E0140020FB
:104B3000DC140020381500201C1500200015002072
:0C4B400004080020081500203415002097
:104B4C0070B5164C164D2B682360FDF7EBFC2B68EB
:104B5C002360144B1D68013D28006B1C17D02D01E0
:104B6C00114BED18114E10E08B420BD1002913D0D4
:104B7C000132A95C935D1C00613C192CF4D8203BDC
:104B8C00DBB2F1E7103D013804D30022F1E701203C
:104B9C00404201E00120404270BDC046AC140020F0
:104BAC00B814002008150020040800205C14002014
:104BBC0010B5FFF7C5FF0400431C0DD002011D4BBF
:104BCC009B18DA68C0231B051A420BD01A4A8023A3
:104BDC0011680B43136010BD174A212311680B4356
:104BEC001360F8E7FFF7ACFF431C11D00201114B27
:104BFC009B18DA68C0231B051A420FD1844213D9C3
:104C0C000C4B24011C19A268000118188260E2E701
:104C1C00094A212311680B431360DCE7064A802301
:104C2C0011680B431360D6E7034A802311680B43CA
:0C4C3C001360D0E70408002024150020BD
:104C480010B5FFF77FFF431C0FD003010D4AD218A0
:104C5800D3681B051B0D0C495B1892689A420AD34E
:104C68000001084A1018836010BD084A2123116802
:104C78000B431360F8E7054A802311680B43136060
:104C8800F2E7C04604080020040200202415002092
:104C9800074B1A68511C196051780902901C18605A
:104CA80092781143802292050A431A607047C046E1
:044CB80018150020AB
:104CBC0010B5084B1B681B68002B08D0064A1368FC
:104CCC0002331360034A1368043B136010BDFFF7F3
:0C4CDC00DDFFF7E7EC14002018150020A5
:104CE80010B5094B1B68191F1A680B689A4208D13E
:104CF800064A136802331360034A1368043B1360BF
:104D080010BDFFF7C5FFF7E7EC14002018150020C9
:104D180010B5094B1B68191F1A680B689A4208DD01
:104D2800064A136802331360034A1368043B13608E
:104D380010BDFFF7ADFFF7E7EC14002018150020B1
:104D480010B5094B1B68191F1A680B689A4208DAD4
:104D5800064A136802331360034A1368043B13605E
:104D680010BDFFF795FFF7E7EC1400201815002099
:104D780030B589B001A80E4B020032CB32C232CB1B
:104D880032C21B88138000F0C0FFFCF727F8002808
:104D9800FBD0FF231840592805D0064800F0B5FF7E
:104DA800002009B030BD0D20FBF7BCFD0120F8E75D
:084DB8006C5E0008D0550008F4
:104DC000F0B58FB0040001A9394B0A0023CB23C2F0
:104DD00023CB23C223CB23C203CB03C2354B1B6897
:104DE0005F2B12D0344D354E33682B60FDF7A0FB9E
:104DF00033682B60FDF73CFC051E10D0304A802341
:104E000011680B431360002506E02D4A8023DB0068
:104E100011680B431360002528000FB0F0BDFDF7AB
:104E200095FC002804D10CA801002A00254F0EE0B3
:104E300001A800F06EFFFFF79FFF0028F3D10225C5
:104E4000EAE7002B12D0072A0AD001320131D35DE4
:104E50000B701E00613E192EF3D8203B0B70F2E759
:104E6000174A022311680B431360D5E70CAB1B787C
:104E7000002B0CD00F4A12681201134952185355D7
:104E800001354378002B02D00130072DF7D1094BB3
:104E90001A6812010C4B9B185D1900226A700B4AAC
:104EA00010680B4A82189A602043D8600125B3E746
:104EB0008455000808150020AC140020B814002008
:104EC000241500205C140020040800203415002064
:044ED00004020020B8
:104ED40070B5C0200005FFF771FF00280DD00A4C03
:104EE40022680A4803681D010949491915688D603B
:104EF400043A22600133036070BD064A80231168BE
:104F04000B431360F8E7C046EC140020081500209A
:084F1400040800202415002010
:104F1C0010B50020FFF74EFF002808D0022807D05C
:104F2C00074B1A68074B1A60074B01221A6010BD19
:104F3C00064B1B681B01064A00219954F7E7C04633
:104F4C0034150020301500202815002008150020ED
:044F5C000408002025
:104F600010B51A4A13681C68043B1360022C1AD847
:104F7000002821D1164800F0CCFE164800F0C9FEEA
:104F800020003030C0B2FBF7D1FC002C18D020201C
:104F9000FBF7CCFC3F20FBF7C9FCFFF7EDFE002838
:104FA00012D0200010BD0C4A8023DB0011680B4397
:104FB000136001246442F4E7084800F0AAFEDCE72D
:104FC000074800F0A6FEE2E70324EAE7EC1400201D
:104FD0009C5F0008B05F000824150020CC5F00082B
:044FE0007C5F0008EA
:104FE40010B50120FFF7BAFF022800D910BD054C07
:104FF4002060FBF747F92368002BF7D0FBF7E2F9B1
:08500400F4E7C0465C15002032
:10500C0010B50020FFF7A6FF02280AD8074B18603E
:10501C00002807D1FFF726FDFBF7F4F8034B00221D
:10502C001A6010BDFBF79AFCFBE7C0465C1500202C
:10503C00074B1B68002B09D0054B00221A60054A50
:10504C001368191D1160044A12685A607047C046F3
:0C505C0040150020EC1400203C15002042
:1050680010B5214B1A68214B1A60FDF75DFAFDF760
:10507800A5FB002821D01C4B1A681C4B1A601C4B3E
:105088001A6812011B4B9B18DA68C0231B051A42C9
:1050980019D0194B1B68002B1BD1184B1B68002B10
:1050A8001AD117480368124A11680901114A52189F
:1050B80019689160043B036004E0124AA023116858
:1050C8000B43136010BD0F4A802311680B43136014
:1050D800F8E7FFF7AFFFE0E76920FDF7D9FB044BDE
:1050E8001868FDF7D5FBEDE7B8140020AC140020D4
:1050F800FC1400200408002020150020281500209A
:08510800EC1400202415002026
:1051100010B5094B1B68002B0BD1084A13680849CE
:1051200018680860043B1360FDF7F4FEFDF768FFA4
:1051300010BDFFF783FFF0E720150020EC140020DE
:0451400038150020FE
:1051440010B5114B1B68002B0DD1104A1368104980
:1051540018680860043B13600E4B1B88DB0705D5F9
:10516400FDF74CFF10BDFFF767FFEEE70A4B1E2269
:105174001A600A4B1968F020400000F0C3FF084B86
:105184001860FDF7C5FEEBE720150020EC140020A5
:10519400001500200004004038150020E41400200D
:0451A4001C150020B6
:1051A80010B5344B1B68002B2FD1334B9B6C01334C
:1051B8002ED0324B1B68002B0DD1314A1360314A77
:1051C80013609023DB051A680F218A431A601A6856
:1051D8000A390A431A602C490B681A682748026082
:1051E800043B0B60002A0AD19023DB05802252027F
:1051F8009A61802292029A611F4B00229A64214B85
:1052080000221A60FDF752FF10BDFFF713FFCCE72D
:105218001A4B00221A609023DB051A680F218A4373
:105228001A601A680A390A431A60174B1A68136811
:10523800002B09DD9023DB05802252029A610222AD
:105248009A61FFF77BFFDFE7002B08DB9023DB0584
:10525800802252029A61802292029A61F1E75B42AF
:1052680013609023DB0501229A61802292029A61E1
:10527800E7E7C0462015002004080020D0140020CD
:0C528800D4140020E8140020EC140020D6
:10529400F0B5C64600B588B069462B4B0A0013CB5F
:1052A40013C213CB13C203CB03C2284B1B68002BBE
:1052B40014D1274A13688024A40519680C43043BBD
:1052C4001360244B9C420CD9234A8023DB001168D1
:1052D4000B43136008B080BCB846F0BDFFF7ACFECA
:1052E400E7E70D20FBF720FB684600F010FD2000E7
:1052F40000F082FE270080370F25032398460FE035
:105304000D20FBF711FB200000F076FE3A20FBF79E
:105314000BFB300000F025FD00250134BC420ED00B
:1053240026780135102DEBD0300000F01AFD4346ED
:105334002B40032BF1D17C20FBF7F6FAEDE70D208F
:10534400FBF7F2FAC6E7C046B05500082015002066
:0C535400EC140020807F002024150020B5
:1053600010B5214B1B68002B34D1204B1B681A68E9
:10537000012A32D9012200241D490A60043B1B493D
:105380000B601C4B5868F0218843586059682143D2
:10539000596053019B1A99008918C900164B186867
:1053A00000F0B2FE013880235B0498420DD2134A0C
:1053B00050601348036A1B021B0AC02109060B43F5
:1053C000036200239360073313600E4B1B68002BAE
:1053D00006D110BDFFF732FEC7E71022B024CBE79D
:1053E000FDF798FDF5E7C04620150020EC140020DD
:1053F000E4140020001002400002002010E000E051
:0854000000ED00E01C15002086
:10540800114B1A6801210A431A605A680F48024072
:105418005A601A680E4802401A601A680D4802401D
:105428001A605A680C4802405A60DA6A0F208243B0
:10543800DA621A6B094802401A635A6B8A435A6344
:1054480000229A607047C046001002400CB8FFF86E
:10545800FFFFF6FEFFFFFBFFFFFFC0FFACFEFFFFF5
:10546800074B1B68002B00DBFEE7054A1168802309
:105478001B060B4313608369023383617047C04680
:045488002CED00E027
:10548C0020286329323032302D323420572E53638A
:08549C0068656D6D6572740016
:0854A4004B65726E656C3A0065
:1054AC00537461636B3D0000436F646554687265AF
:1054BC0061643D00456D7074795F000050726F6AD5
:1054CC006563740020204155544F4558453D0000FC
:1054DC002020204C45446D6F64653D002020204306
:1054EC005055636C6F636B3D000000004261756446
:1054FC00526174653D0000002870656E64696E67CA
:10550C00290000002020465245513D00487A205089
:10551C00574D313D000000002020204D4F543A00E3
:10552C00537465703D0000006D73204E5354503D14
:0C553C000000000044432F50574D310088
:10554800416374697665206174206E6578742053B0
:0C555800797374656D20537461727400E7
:10556400243800087A3800088C3800089E3800086F
:10557400B0380008C2380008D438000800390008E0
:10558400205761726E3A2077696C6C206F76657271
:1055940072696465204B65726E656C204F5020778C
:0C55A4002E73616D65206E616D65200046
:1055B000313238205352414D206279746573207323
:1055C00074617274696E672066726F6D2030780046
:0C55D0002063616E63656C6C65642000F4
:1055DC0000000000000000000000000000000000BF
:1055EC0000000000000000000000000000000000AF
:1055FC00000000000000000000000000000000009F
:10560C00000000000000000000000000000000008E
:10561C00000000000000000000000000000000007E
:10562C00000000000000000000000000000000006E
:10563C00000000000000000000000000000000005E
:10564C00000000000000000000000000000000004E
:10565C00000000000000000000000000000000003E
:10566C000000000000000000000001000000050028
:10567C00000000000000000000000000000000001E
:10568C00000000000000000000000000000001000D
:10569C0000000400000004000000000000000000F6
:1056AC0000000000000000000000000000000000EE
:1056BC0000000400000004000000040000000000D2
:1056CC0000000000000000000000000000000000CE
:1056DC0000000000000000000000000000000000BE
:1056EC0000000400000000000000050000000500A0
:1056FC00000005000000040000000400000004008D
:10570C000000040000000000000001000000010087
:10571C000000010000000100000003000000030075
:10572C000000030000000300000003000000030061
:10573C000000030000000300000003000000030051
:10574C000000030000000300000002000000020043
:10575C000000020000000200000002000000010036
:10576C000000010000000800000008000000080014
:10577C0000000800000008000000080000000800FD
:10578C0000000800000008000000080000000800ED
:10579C0000000800000008000000080000000800DD
:1057AC0000000800000002000000020000000100E0
:1057BC0000000100000000000000040000000500D3
:0857CC000000010000000100D3
:1057D4004552524F5200000044524F500000000006
:1057E4004455500000000000535741500000000091
:1057F4004F56455200000000524F54000000000074
:105804002D524F54000000005049434B000000004B
:10581400524F4C4C00000000494E4A45435400008E
:105824002B00000000000000312B000000000000ED
:105834002D00000000000000312D000000000000D9
:105844004142530000000000534849465400000000
:10585400414E4400000000004F52000000000000D0
:10586400584F5200000000004E4F5400000000004A
:105874002B2F2D00000000002A0000000000000073
:105884002F000000000000002A2F0000000000008C
:105894004D4F4400000000002F4D4F440000000015
:1058A400425345540000000042434C5200000000A3
:1058B400425453540000000052414E444F4D0000E6
:1058C4003D3D000000000000213D000000000000FC
:1058D4003E000000000000003E3D0000000000000B
:1058E4003C00000000000000553C000000000000E7
:1058F4003C3D000000000000303D000000000000BE
:10590400564152434F4E00005245560000000000DD
:1059140041525241590000004B45593F00000000DC
:105924004B45590000000000454D4954000000005B
:105934002E000000000000002E48000000000000BF
:105944002E440000000000002E2200000000000091
:10595400445A000000000000485800000000000005
:10596400584E4F50000000004D530000000000004E
:105974004453000000000000544958000000000097
:1059840054494D4500000000534C4545500000006B
:10599400465245510000000050574D3100000000B0
:1059A4004D4F5400000000004F480000000000006C
:1059B4004F4C00000000000049505500000000005A
:1059C4004950440000000000495A00000000000053
:1059D4005244494E0000000052414443000000007C
:1059E400494E492D535049005350490000000000CE
:1059F4002E53000000000000465300000000000089
:105A04004F50530000000000555345520000000061
:105A140053454500000000004D454D0000000000C6
:105A2400535400000000000052554E0000000000D6
:105A34004E4F2D4442470000444542554700000064
:105A4400464F52474554000041424F525400000013
:105A54005245504C41434500524553544F52450022
:105A64004946000000000000434153450000000087
:105A74003C434153450000003E4341534500000070
:105A8400454C5345000000005448454E00000000BA
:105A9400444F000000000000554E54494C000000E3
:105AA4005748494C45000000414741494E00000019
:105AB400464F5200000000004C4F4F5000000000C1
:105AC4004900000000000000434F4E54490000000C
:105AD400425245414B0000005A425245414B00009E
:105AE40052455455524E00003A0000000000000098
:105AF4003B00000000000000646F5354520000009B
:105B0400646F4C4954384200646F4C49540000009F
:105B1400646F56414C554500646F52455600000071
:105B2400646F494600000000646F43415345000020
:105B3400646F3C4341534500646F3E434153450009
:105B4400646F454C53450000646F444F00000000EF
:105B5400646F554E54494C00646F5748494C450096
:105B6400646F414741494E00646F464F5200000044
:105B7400646F4C4F4F50000052502D310000000014
:105B840052502D34000000004155544F45584500F3
:105B940042415544000000004C4544000000000010
:105BA40053504545440000003F0000000000000041
:105BB40053415645000000004C4F41440000000092
:105BC400FEE7FEE7FEE7FEE7FEE7FEE7FEE7FEE7A9
:105BD400FEE7FEE7FEE7FEE7FEE7FEE7FEE7FEE799
:105BE400FEE7FEE7FEE7FEE7FEE7FEE7FEE7FEE789
:105BF400FEE7FEE7FEE7FEE7FEE7FEE7FEE7FEE779
:105C0400FEE7FEE7FEE7FEE7FEE7FEE7FEE7FEE768
:105C1400FEE703488546FFF7F5FB03E07047000005
:045C24000018002044
:105C280011488546114C20680434004201D0804751
:105C3800F9E70F480F49091A082903DB0022026017
:105C4800043001600C480D49884205D002680430D0
:105C580003B4904703BCF7E700208646EC460020D3
:105C68000021074A9047FEE70018002070610008ED
:105C780078150020C0160020C55E0008C55E000823
:045C88007D0C000887
:105C8C0004207146084202D1EFF3088001E0EFF3E3
:0C5C9C0009800149084700006954000815
:105CA80043466F727468204C6F77506F7765722D1A
:105CB80034384D487A2F334D487A2C6E6F555342FD
:105CC8002D20666F722053544D33324630343220C3
:025CD800760054
:0A5CDA003323013B002BFCD170477F
:105CE400756E646572666C6F77212000202D2D2DF2
:025CF40020008E
:105CF60010B502003030C0B2392801D93732D0B2DF
:065D0600FAF711FE10BDCA
:065D0C002849502D3E0065
:105D120010B5441C0078002806D0FAF706FE0134BC
:0A5D2200631E18780028F8D110BDA8
:105D2C0063616E277420534545204B65726E656C1C
:105D3C00204F7073000000005573657248656164F4
:105D4C0065725F5374727563743D000056617243E3
:0A5D5C006F6E3A56616C75653D00EC
:105D660010B5040003061B0F18003030392801D97E
:105D760037331800FAF7D7FD0F20044020003030E3
:105D8600392800D90730FAF7CEFD2020FAF7CBFDE7
:025D960010BD3E
:105D98004572726F722300002028636F6C20000028
:105DA800206E6F7420666F756E6400005F53796EA5
:105DB80074617820457272005F537461636B20458B
:105DC800727200005F436F6D70696C65206F6E6C56
:105DD800790000005F496E76616C696420436F64E6
:105DE8006520616363657373000000005F6F7574FD
:105DF800206F6620436F6E74657874005F52756E0D
:105E080074696D65206F6E6C790000005F5468726C
:105E18006561642063616E63656C6C656400000095
:105E28005F4E756D626572206F7574206F662052C3
:105E3800616E6765000000005F4469762E62792014
:105E48005A65726F000000002020636F6D70696CE6
:065E5800696E672E2E00AA
:0E5E5E0010B5FAF73EFE2020FAF761FD10BDE8
:105E6C0020636F6E6669726D20772E757070657227
:0A5E7C002063617365202759270099
:105E86002F280FD90300303BDBB2092B08D90A298A
:105E96000BD00300413B052B0AD83738C0B27047F8
:105EA6001800FCE701204042F9E701204042F6E7EE
:065EB60001204042F3E769
:095EBC0028566172436F6E3D002F
:0E5EC60010B56A20FCF7E5FCFDF735FE10BDB7
:105ED400203C2D6E6F742061204B65726E656C20C2
:105EE4004F50206E6F722061206E756D6265720076
:105EF400203C2D696E76616C696420666F72204265
:105F040061636B2D4374726C00000000203C2D52C1
:0D5F1400756E74696D65204572726F7200C4
:0E5F220010B56B20FCF7B7FCFDF707FE10BDB5
:105F300020202841444320696E6974292000000014
:0D5F4000202028414443206F666629200080
:0E5F4E0010B56C20FCF7A1FCFDF7F1FD10BDB5
:105F5C002064656275672066696E69736865642084
:015F6C000034
:0E5F6E0010B56D20FCF791FCFDF7E1FD10BDB4
:105F7C00283D456D7074792050726F6A6563742981
:015F8C000014
:0E5F8E0010B57020FCF781FCFDF7E5FD10BD9D
:055F9C004C6F61640080
:0E5FA20010B57120FCF777FCFDF7DBFD10BD9C
:0D5FB0002050726F6A656374206E6F2E00C2
:0E5FBE0010B57220FCF769FCFDF7CDFD10BD9B
:055FCC00536176650041
:105FD2000A0010D00300400800E052008242FCD9BF
:105FE200002000E05208934200D39B1A40418A42AB
:0A5FF200F8D1190070470020704735
:105FFC0070B50400000FFFF778FE200E0F25284027
:10600C00FFF773FE200D2840FFF76FFE200C284091
:10601C00FFF76BFE200B2840FFF767FE200A284095
:10602C00FFF763FE20092840FFF75FFE28002040A1
:0C603C00FFF75BFE2020FAF773FC70BD3C
:1060480010B50400000F16D12001000F17D120024F
:10605800000F18D12003000F19D12004000F1AD106
:106068002005000F1BD12006000F1CD10F20204057
:10607800FFF73DFE10BDFFF73AFE2001000FFFF7C6
:1060880036FE2002000FFFF732FE2003000FFFF755
:106098002EFE2004000FFFF72AFE2005000FFFF751
:0C60A80026FE2006000FFFF722FEDFE7B7
:1060B40010B504003020FAF737FC7820FAF734FCE6
:0860C4002000FFF7BFFF10BD33
:1060CC00CA1751408B1A17D0C1174A4004B4484024
:1060DC00411A48081A0000E052008242FCD9002004
:1060EC0000E05208914200D3891A40419A42F8D1FB
:0C60FC0004BC5040801A70470020704720
:106108000A000FD00300400800E052008242FCD988
:10611800002000E05208934200D39B1A40418A4273
:08612800F8D170470020704718
:10613000CA1751408B1A19D0C11706B44840411AEA
:1061400048081A0000E052008242FCD9002000E01A
:106150005208914200D3891A40419A42F8D10CBCAE
:1061600053405840C01A5140891A70470020704768
:10617000956300080402002071130000AB6300085F
:1061800000000020906100080402000000000000F0
:106190002D0F00083D0F0008650F0008950F00083F
:1061A000AD0F0008C10F0008E50F00080910000836
:1061B00049100008A910000809110008251100085D
:1061C000351100085111000861110008791100080B
:1061D000C1110008DD110008F911000815120008AE
:1061E0002512000835120008511200088912000813
:1061F000C1120008F91200083913000871130008D1
:10620000A9130008E5130008FD1300081D14000879
:10621000511400087514000899140008BD140008F2
:10622000DD1400083D140008D54E00086950000830
:1062300001150008452D0008B51A0008291A0008A4
:10624000111B0008591B0008411D00082D2E0008D5
:10625000551500087515000895150008E53100086A
:1062600095320008B1150008CD150008B1360008B8
:106270001151000845510008A95100085D3300087C
:10628000F1330008893400081135000899350008F9
:10629000DD320008A1370008C9390008053A0008B6
:1062A000791B0008E9160008591D00083D1C00086C
:1062B000D142000895520008091700081517000878
:1062C00021170008411A000865460008DD4600084D
:1062D000BD4B0008494C0008C75E0008235F00085A
:1062E0004F5F00086F5F00087D2A0008ED15000869
:1062F000C52A00088F5F0008A35F0008BF5F000881
:10630000F12A00081D2B0008211600085D1800085E
:106310003D16000851160008791600081D4F0008A8
:10632000752B0008851A00086D1700082D17000846
:106330008D170008B9170008BD4C0008E94C00088B
:10634000194D0008494D0008E51700080918000814
:106350008D180008C518000839180008FD18000835
:106360004D190008D9190008E9190008412800084A
:10637000AD220008F919000861530008F11D00085A
:10638000E54F00080D500008010000001413002024
:04639000006CDC02BF
:10639400206861680834094204D000220270013088
:0663A4000139FBD1704736
:1063AA0020686168A2680C34124205D00B78037029
:0A63BA0001300131013AF9D17047BA
:0400000508005C177C
:00000001FF
